:03000000023421A6
:0C34210078FFE4F6D8FD75815402346891
:1012FD0020000A3C2E2E2E3E004950436F6E6E6527
:10130D0063745245510A004950436F6E6E656374A4
:10131D00000A49504E6F41434B210A003E432C5663
:10132D002C52432CC0E4E0EFF2E5F020D1E8EDEAD9
:10133D00EEEC49500A003E432C4D41432C253032F2
:10134D0062583A25303262583A25303262583A2581
:10135D00303262583A25303262583A25303262586E
:10136D002C4D414320E0E4F0E5F10A003E432C56BC
:10137D0045522C20332E3220EEF22025732025737A
:10138D002CC2E5F0F1E8FF20495020ECEEE4F3EB40
:10139D00FF0A004170722032352032303038003172
:1013AD00363A31363A3230003E432C4C442C5052B2
:1013BD004F473A20202020202020202020202020B0
:1013CD002020202020202020202020202020202010
:1013DD002020202020202020202020202020202000
:1013ED0020202020202020202020202020202020F0
:1013FD0020202020202020202CC4E0F2E020EFF03F
:10140D00EEF8E8E2EAE828F4E0E9EB290A003E2AE2
:10141D002C312CCEF1EDEEE2EDFBE520EFE0F0E02E
:10142D00ECE5F2F0FB20F1E5F2E5E2EEE3EE20E88B
:10143D00EDF2E5F0F4E5E9F1E00A003E412C413032
:10144D00312C2562752E2562752E2562752E25622D
:10145D00752C495020E0E4F0E5F120E0E4E0EFF2F6
:10146D00E5F0E00A003E412C4130322C2562752E0C
:10147D002562752E2562752E2562752C495020E04A
:10148D00E4F0E5F120EEF1ED2E20F1E5F0E2E5F0EE
:10149D00E00A003E412C4130332C2562752E256229
:1014AD00752E2562752E2562752C495020E0E4F0CD
:1014BD00E5F120F0E5E72E20F1E5F0E2E5F0E00AB8
:1014CD00003E412C4130342C2562752E2562752E3F
:1014DD002562752E2562752CCCE0F1EAE020F1E550
:1014ED00F2E80A003E412C4130352C2562752E253F
:1014FD0062752E2562752E2562752CD8EBFEE70AD6
:10150D00003E2A2C312CC4EEEF2E20EFE0F0E0EC63
:10151D00E5F2F0FB20F1E5F2E5E2EEE3EE20E8ED99
:10152D00F2E5F0F4E5E9F1E00A003E422C533031EA
:10153D002C2562752CC6E4E0F2FC20E7E0EFF0EE1E
:10154D00F1E020F1EEE5E4E8EDE5EDE8FF20EEF267
:10155D0020F1E5F0E2E5F0E00A003E422C53303296
:10156D002C2562752CCEE1ECE5ED20F120F1E5F0B6
:10157D00E2E5F0EEEC20E1E5E720EAE2E8F2E0ED6D
:10158D00F6E8E90A003E422C5330332C2562752CC7
:10159D00CFE5F0E5E7E0EFF3F1EA20EFF0E820EF3B
:1015AD00EEF2E5F0E520F1E2FFE7E820F120F1E5CC
:1015BD00F0E2E5F0EEEC0A003E454E440A000A4426
:1015CD00756D705820202020203030203031203093
:1015DD003220303320303420303520303620303733
:1015ED002030382030392030412030422030432007
:1015FD003044203045203046000A3A003A20000A97
:10160D00000A44756D704420202020203030203099
:10161D0031203032203033203034203035203036F8
:10162D0020303720303820303920304120304220D2
:10163D003043203044203045203046004572722022
:10164D006B657900526420656570726F6D0A00528A
:10165D0064204D454D0A00526420436F64650A00B5
:10166D00577269746520436F64650A00446562753D
:10167D00674950204F4E0A004465627567495020F6
:10168D004F46460A00446562756755736572204F73
:10169D006E0A00446562756755736572204F464644
:1016AD000A0044656275674D7367204F6E0A0044EA
:1016BD00656275674D7367204F46460A00436F6E2E
:1016CD00666967206C6F636B210A00577220656530
:1016DD0070726F6D0A0020536176652065657072BA
:1016ED006F6D210A00457272204D414321004C6FF0
:1016FD0061643E3E002A003C4130313D003C4130AA
:10170D00323D003C4130333D003C4130343D003CE6
:10171D004130353D003C21003C5330313D003C53C0
:10172D0030323D003C5330333D003C5330353D00AD
:06173D003C5330363D0074
:063CAB00015100014F0071
:103CF500C28E438910E4F58B758DB8D2ABD28E2276
:03001B000233911C
:10339100C0E0C083C082C0D0C28E758B00758DB86D
:1033A100201D0675A61E75A6E1054FD219E55160CF
:1033B100020551E550D39401400215500554E554DE
:1033C100540F7048D225E554543F7012D2179066BD
:1033D1008BE0600A04F0E0D394B44002D21D906601
:1033E10086E0600204F0906104E0600214F09066EF
:1033F1008CE0D394014003E014F0301C020552E547
:1034010053D394644004D21D80020553E54ED394F6
:10341100014002154ED28ED0D0D082D083D0E0327E
:10084F00C2AFC2227D027C007F07123C8E8F26E54D
:10085F0026646060097D017F60123C26D222E4FD90
:10086F00FC7F0B123C8E8F26E52630E6097D04E4D3
:10087F00FF123C4AD2227D017C007F07123C8E8FF3
:10088F0026E5267008FD7FFF123C26D22230220378
:10089F00126000C288C2A8C2AA7589001232F590F0
:1008AF0063497403F0A374CCF0E4906348F0122F03
:1008BF00681230EEC21D123956D222C224C22390C2
:1008CF0065767408F09062B47424F0E4A3F090633A
:1008DF003EE09062B6F090633FE09062B7F09063B5
:1008EF0040E09062B8F0906341E09062B9F090639D
:1008FF0042E09062BAF0906343E09062BBF07550B3
:10090F0001E4906577F0C21EC21FC220C2212022CF
:10091F0018AF26FE7D03122DACE4FF1231A27E121A
:10092F007FFDE4FBFDFC1228CC90668BE060037426
:10093F0001F0E4906104F0F552906575F0F55312F3
:10094F003CF575A70775A61E75A6E1D2AFE4F55362
:10095F00906104E07003123A0690668CE0B40111C6
:10096F009080007410F0E490668CF0D222C223C203
:10097F0024908008E0F52630E405D21E7410F0E5CF
:10098F002630E508D2209080087420F0E52630E666
:10099F0008D21F9080087440F0E552C394034019A9
:1009AF00908002E4F0908001F0908000F0E5529486
:1009BF00064006E4F5521239569080A0E0700312FB
:1009CF0037499080B8E070031237C39080D0E07041
:1009DF000312383D908000E07013301E101229D39F
:1009EF00906331EFF0D39400400312002690800201
:1009FF00E07006908000E06005D21C02095CC21C0A
:100A0F00E4F552906104E0600302095C2022129029
:100A1F006578E0600C7E127FFF122CC4E49065783D
:100A2F00F0302012122612906331EFF0D394004071
:100A3F0005E0FF123D62201F03020BC012248B90B2
:100A4F006331EFF0700302095C906375E054BF24CB
:100A5F007F7003020B29147003020B012402600341
:100A6F00020B622022077E137F06122CC42026035E
:100A7F00020BC090634DE0FF7006906351E0606120
:100A8F00906682E0FEB50722A3E0FF90634EE0B5CB
:100A9F000718906684E0FF90634FE0B5070C9066EF
:100AAF0085E0FF906350E06F6037906351E06E60B8
:100ABF0003020BC0906683E0FF906352E06F600308
:100ACF00020BC0906684E0FF906353E06F600302F7
:100ADF000BC0906685E0FF906354E06F6003020BDC
:100AEF00C0C21A9065777401F012001E7550010292
:100AFF000BC090668BE060037401F090667AE0FFA4
:100B0F00906377E06F6003020BC090667AE004F0A9
:100B1F00E4F550906575F0020BC0301A03020BC05C
:100B2F00906344E0700302095C906355740AF012FD
:100B3F003D49D21AE4F550906575F090668604F041
:100B4F00E4906679F0A3F02022677E137F14122CB5
:100B5F00C4805E90668BE060037401F0301A52908F
:100B6F006375E020E74B906377E0FF906679E0FED6
:100B7F006F600D906681E07007EE146F7033801315
:100B8F00906679E004F0906331E0FFD39404400362
:100B9F001239AF9060007482F0A37401F090637704
:100BAF00E0906002F07E607F007D03123534020911
:100BBF005C201A03020CD8E55070681222F7EF6020
:100BCF00237E647F75906476E02404FD12353490A3
:100BDF006681E07009906355E0F55002095CE4F519
:100BEF005002095C906686E0D3943C403690668153
:100BFF00E0703090668604F0123032E4906475F045
:100C0F00A37412F090667AE0906477F0A374FDF00D
:100C1F0090610563A20190647963A2017F12122093
:100C2F0045809E123D148F26E526B4011590600075
:100C3F007483F0E4A3F07E607F007D0212353402EE
:100C4F00095CE526D39401401C9060007483F0A3E7
:100C5F007401F0E52624FEA3F07E607F007D031271
:100C6F00353402095CE5506401600302095C90654C
:100C7F0075E004F02022077E137F1E122CC49063B0
:100C8F0055E0C394C85004E02432F0906575E0C37A
:100C9F009405400DC21AE4906577F012001E020908
:100CAF005C7C667D82906349E0FAA3E0FB7F0212D1
:100CBF0036C57E647F75906476E02404FD1235346A
:100CCF00906355E0F55002095CE550640160030242
:100CDF00095C906577E014604624FE60421470034F
:100CEF00020DCB2404600302095CE4F552202613A5
:100CFF009065777404F0906575E05401F0755001BC
:100D0F0002095C9080027410F0E4906577F09065B2
:100D1F007504F07550FA90668274FFF002095C90CA
:100D2F006682E07003020DB59064757480F0906474
:100D3F00777401F0E4A3F0A304F0A37430F0A3746C
:100D4F007BF0E4F526747C2526F582E43464F58384
:100D5F00747DF0747D2526F582E43464F583E4F028
:100D6F00E5262407906476F07C667D82906349E0E7
:100D7F00FAA3E0FB7F021236C57E647F75E5262459
:100D8F0009FD123534906681E0601B123D49D21A7D
:100D9F00E4F550906575F090668604F0E4906679FE
:100DAF00F0A3F002095C302607E4906577F0800627
:100DBF009065777404F07550FA02095C90800274A4
:100DCF0010F0755005906575E06401FFF090657740
:100DDF007401F0EF7019906351E06013FCA3E0FD14
:100DEF00A3E0FEA3E0FF906682121BE402095C9071
:100DFF00634DE0FCA3E0FDA3E0FEA3E0FF9066825D
:090E0F00121BE402095C80FE22C2
:10002600906376E0B444047F0180027F009063759C
:10003600E0B447047E0180027E00EE5F604A906372
:100046003EE0906377F090633FE0906378F09063D2
:1000560040E0906379F0906341E090637AF09063BA
:1000660042E090637BF0906343E090637CF09063A2
:10007600767452F09062AE63A2019080A863A201EA
:100086007F06122045020845906331E0C39408506C
:100096000302084E90633EE0FF906377E06F6003D3
:1000A60002084E90633FE0FF906378E06F600302C2
:1000B600084E906340E0FF906379E06F60030208AA
:1000C6004E906341E0FF90637AE06F600302084E52
:1000D600906342E0FF90637BE06F600302084E90FE
:1000E6006343E0FF90637CE06F600302084E906319
:1000F60076E0B444159062AEE0B4FF0E63A20190C0
:1001060080A863A2017F0612204590668BE06003FB
:100116007401F090668C7464F09063767452F0907B
:100126006375E0646D60030202537BFF7A137929DD
:100136001217A57BFF7A13794390633EE0F52FA350
:10014600E0F530A3E0F531A3E0F532A3E0F533A303
:10015600E0F5341217A5752FFF7530137531A075AC
:1001660032FF7533137534AC7BFF7A137979121726
:10017600A57BFF7A1379B51217A57BFF7A14791B35
:100186001217A57BFF7A147948906344E0F52FA3F4
:10019600E0F530A3E0F531A3E0F5321217A57BFFB9
:1001A6007A14797290634DE0F52FA3E0F530A3E061
:1001B600F531A3E0F5321217A57BFF7A1479A090EA
:1001C6006351E0F52FA3E0F530A3E0F531A3E0F5A8
:1001D600321217A57BFF7A1479CE90633AE0F52F99
:1001E600A3E0F530A3E0F531A3E0F5321217A57BC5
:1001F600FF7A1479F1906336E0F52FA3E0F530A38A
:10020600E0F531A3E0F5321217A57BFF7A15790EDA
:100216001217A57BFF7A157937A226E433F52F123C
:1002260017A57BFF7A157967906681E0F52F12177F
:10023600A57BFF7A15799290668BE0F52F1217A5AC
:100246001232527BFF7A1579C51217A52290637573
:10025600E0644C70737E157FCBFBFDFC1228CC90BE
:10026600637DE0F527A3E0F528E4F52AE52790630A
:100276007FF0A3E528F07E167F067C637D7F7B02F8
:100286001228CCE4F529852882852783E0FF747F30
:100296002529F582E43463F583EFF00528E5287017
:1002A6000205270529E529B410DC7E167F097C6343
:1002B6007D7F7B101228CC052AE52AC3941040AC1A
:1002C6007E167F0C122CC422906375E0646C7060FD
:1002D600F52B7E167F0EFBFDFC1228CCE4F52AE4F6
:1002E60090637FF0A3E52BF07E167F067C637D7F0F
:1002F6007B021228CCE4F529A82BE6FF747F25297A
:10030600F582E43463F583EFF0052B0529E529B47E
:1003160010E67E167F097C637D7F7B101228CC0554
:100326002AE52AC3940840B77E167F0C122CC422F5
:10033600906375E0644B7061F52974672529F58231
:10034600E43463F583E0603274672529F582E4348A
:1003560063F583E0F4602374672529F582E434634A
:10036600F583E0FF747D2529F582E43463F583E0A7
:10037600B507100529E529B408C09061047432F068
:100386000208459063757421F03022030208457E09
:10039600167F49122CC4020845906375E0B4521AC0
:1003A6002022077E167F51122CC49063757472F05A
:1003B6007E637F757D081234AD22906375E06449D3
:1003C60070452022077E167F5C122CC490637DE068
:1003D600F527A3E0F528E4F529852882852783E01B
:1003E600FF747F2529F582E43463F583EFF0052851
:1003F600E528700205270529E529B480DC7E637FA0
:10040600757D8A1234AD22906375E0644370462090
:1004160022077E167F64122CC490637DE0F527A325
:10042600E0F528E4F529852882852783E493FF747F
:100436007F2529F582E43463F583EFF00528E52866
:10044600700205270529E529B480DB7E637F757D6B
:100456008A1234AD22906375E0645A7053202207E5
:100466007E167F6D122CC490637DE0F527A3E0F520
:10047600287C637D7F7B80AF28AE27123B4CE4F55A
:1004860029852882852783E493FF747F2529F582B1
:10049600E43463F583EFF00528E5287002052705A7
:1004A60029E529B480DB7E637F757D8A1234AD220F
:1004B600906375E06444600302054790637DE0FF46
:1004C60064447003020845EFB4310CC2227E167FE5
:1004D60079122CC402084590637DE0B4300CD22218
:1004E6007E167F85122CC402084590637DE0B432E7
:1004F6000CD2237E167F92122CC402084590637D8F
:10050600E0B4330CC2237E167FA0122CC402084529
:1005160090637DE0B4340CD2247E167FAF122CC4D7
:1005260002084590637DE0B4350CC2247E167FBC7C
:10053600122CC402084590637DE0FF123D6102085B
:1005460045906104E070132022077E167FCA122CA4
:10055600C49063757421F00208459061047432F00A
:10056600906375E0FFB45104C2AF80FEEF6457702C
:10057600452022077E167FD8122CC490637EE09019
:100586006331F0E4F529906331E0FFE529C39F402C
:1005960003020845747F2529F582E43463F583E078
:1005A600FF90637DE0252924ADF582E43461F5836F
:1005B600EFF0052980D0906375E06453600302066E
:1005C600692022077E167FE3122CC490633EE0FF6B
:1005D6009061B6E06F703C90633FE0FF9061B7E0DA
:1005E6006F7030906340E0FF9061B8E0B5072490EB
:1005F6006341E0FF9061B9E0B50718906342E0FF00
:100606009061BAE0B5070C906343E0FF9061BBE0F0
:100616006F60169063757421F03022030208457EE0
:10062600167FF2122CC4020845E4F529E4F553744A
:10063600AD2529F582E43461F583E0FDAF29123B4F
:10064600AC0529E529C394FE40E2C2AFE4907FF0F1
:10065600F0A3F0907FFD74AAF0A374FFF0A3745585
:10066600F080FE906375E0644F704C90637DE0F51A
:1006760027A3E0F528E5284527700A2022077E16DD
:100686007FFB122CC42022077E177F02122CC4E4A3
:10069600F529747F2529F582E43463F583E08528FE
:1006A60082852783F00528E528700205270529E5B8
:1006B60029B480DE020845906375E0FFB4452190B9
:1006C600637DE0FDA3E0907FF0CDF0A3EDF0C2AF37
:1006D600907FFD74AAF0A374FFF0A37455F080FE1A
:1006E600EF6465600302084E90637DE0FFA3E0902F
:1006F6007FF0CFF0A3EFF0E4F527F528D3907FF154
:10070600E09528907FF0E095274021E4F5532528D1
:10071600FFE5273478FE7B80AD28AC27123B4C746E
:10072600802528F528E43527F52780D07E177F0415
:100736001235BBEF4E6020120003906344EFF012B7
:100746000003906345EFF0120003906346EFF0124A
:100756000003906347EFF07E177F0A1235BBEF4E1A
:10076600602012000390634DEFF012000390634E79
:10077600EFF012000390634FEFF012000390635006
:10078600EFF07E177F101235BBEF4E60201200038C
:10079600906351EFF0120003906352EFF0120003E2
:1007A600906353EFF0120003906354EFF07E177FCF
:1007B600161235BBEF4E602012000390633AEFF03D
:1007C60012000390633BEFF012000390633CEFF0DE
:1007D60012000390633DEFF07E177F1C1235BBEFCE
:1007E6004E6020120003906336EFF0120003906310
:1007F60037EFF0120003906338EFF01200039063B6
:1008060039EFF0E4F529E4F553E52904FF743625BC
:1008160029F582E43463F583E0FD123BAC0529E556
:1008260029C3944340E0C2AFE4907FF0F0A3F09078
:100836007FFD74AAF0A374FFF0A37455F080FE7ECA
:09084600637F757D081234AD22B8
:103ADE00AE07EEC39430400BEED394395005EE246E
:103AEE00D0FF22EEC39461400BEED394665005EEE8
:103AFE0024A9FF22EEC39441400BEED39446500509
:083B0E00EE24C9FF22AF0622DC
:103CC7009062ADE004F070069062ACE004F09062A0
:0A3CD700ACE0FEA3E0FF123A9C22CD
:10000300123CC7123ADEEFC454F0FEC006123CC7DE
:08001300123ADED0E02FFF22BB
:1038A000E49069C2F0123CC79069C3EFF0C3943052
:1038B0004018E0FFD3943950119069C2E02405F517
:1038C00082E43461F583EFF080119069C2E0240551
:1038D000F582E43461F583E4F0800C9069C2E00481
:1038E000F0E0D3940840BE753200753300753400A3
:0D38F000E4F5357B017A6179051221532240
:1035BB008E2C8F2D9062ACE4F0A374FFF0123CC7FD
:1035CB00EF606EF4606B852D82852C83E493B507D9
:1035DB00EC752E01E52D252EF582E4352CF583E4D3
:1035EB009360259062ADE0252EFF9062ACE0340035
:1035FB00FE123A9CE52D252EF582E4352CF583E45D
:10360B0093B50704052E80CCE52D252EF582E435E8
:10361B002CF583E49370A6E52E24FFFFE434FFFE24
:10362B009062ADE02FF09062ACE03EF07E007F0147
:05363B0022E4FEFF2265
:102F68007E177F221235BBEF4E70037F01227E173A
:102F78007F251235BBEF4E600C123CC7EF24D024DE
:102F8800FF92268002D2267E177F2B1235BBEF4E8A
:102F9800600C123CC7EF24D0906681F08005E49065
:102FA8006681F07E177F311235BBEF4E600C123C04
:102FB800C7EF24D090668BF08005E490668BF07E96
:102FC800177F371235BBEF4E600C123CC7EF24D089
:102FD80024FF92188002C21890633E63A201906693
:102FE8007B63A2017F0612204530183B7E177F3D88
:102FF8001235BBEF4E603012000390667BEFF01283
:10300800000390667CEFF012000390667DEFF012EB
:10301800000390667EEFF012000390667FEFF012D7
:0A3028000003906680EFF07F0022A5
:103A5500906576E0C3947C503D906576E0FE04F079
:103A650074B42EF582E43462F583EFF0BF0A279033
:103A75006576E0FF04F074B42FF582E43462F583D3
:103A8500E4F0906576E0FF1236409065767408F0B4
:073A95009062B5E004F0228D
:100E18005452414E5A0053545245414D0052545376
:100E28000044454C4159004D4F4445004C494D49FB
:100E3800540053495A45004C454E475448004556BE
:100E4800454E504152495459004F4444504152492B
:100E58005459004B56545F494E004B56545F4F55FA
:100E68005400574149540053544F5000003E2A2C17
:100E7800312CCFE0F0E0ECE5F2F0FB20E0F1E8ED1A
:100E8800F5F0EEEDEDEEE3EE20EFEEF0F2E02E20E1
:100E9800D0E5E6E8EC20F0E0E1EEF2FB202D20EFD3
:100EA800E0EAE5F2EDFBE90A003E4C2C4930312C32
:100EB800256C752CD1EAEEF0EEF1F2FC20EEE1ECB7
:100EC800E5EDE02C35302C3130302C3330302C36F9
:100ED80030302C313230302C323430302C34383001
:100EE800302C393630302C31393230302C333834DC
:100EF80030302C35373630302C3131353230300AFD
:100F0800003E422C4930322C2562752CD3EFF0E09C
:100F1800E2EBE5EDE8E520EFEEF2EEEAEEEC20EFAD
:100F2800F0E820EFE5F0E5E4E0F7E5202852545337
:100F38002D435453290A003E532C4930332C256243
:100F4800752CC7E0E4E5F0E6EAE020F1F2E0F0F223
:100F5800E020EFE5F0E5E4E0F7E8282A3130ECF1AD
:100F6800290A003E422C4930342C2562752CD0E5E4
:100F7800E6E8EC20EFE5F0E5E4E0F7E8203720E1EB
:100F8800E8F20A003E422C4930352C2562752CCFF8
:100F9800E5F0E5E4E0F7E020F120EAEEEDF2F0EE2E
:100FA800EBFCEDFBEC20E1E8F2EEEC0A003E422C13
:100FB8004930362C2562752CCAEEEDF2F0EEEBFCCA
:100FC800EDFBE920E1E8F2202D20F7E5F2EDEEF166
:100FD800F2FC0A003E422C415030372C2562752C19
:100FE800C6E4E0F2FC20EAE2E8F2E0EDF6E8FE20F2
:100FF800EEF220F3F1F2F0EEE9F1F2E2E00A003E5F
:10100800422C415030382C2562752CCAE2E8F2E8AF
:10101800F0EEE2E0F2FC20EFE0EAE5F2FB20EEF28F
:1010280020F3F1F2F0EEE9F1F2E2E00A003C2100EF
:101038003C4930313D003C4930323D003C49303379
:101048003D003C4930343D003C4930353D003C4989
:1010580030363D003C415030373D003C415030383F
:101068003D000A53656E64205061636B65743A20D5
:10107800000A53656E64204B56543A20000AC1F3A7
:10108800F4E5F020E7E0EDFFF221000A43524320A7
:101098006572726F7221202020000ACEF2E2E5F715
:1010A800E0FE20EDE020E7E0E3F0F3E7EAF32100DB
:1010B8000A526563204B5654000A526563206F6BD1
:1010C8002120202020202000FF0E18FF0E1EFF0EDA
:1010D80025FF0E29FF0E2FFF0E34FF0E3AFF0E3F9D
:1010E800FF0E46FF0E51FF0E5BFF0E62FF0E6AFFFA
:1010F8000E6FFF0E7400112332465765748C9DAF36
:10110800BECADBE9F810013322564775649C8DBFCF
:10111800AEDACBF9E82130021367764455ADBC8EC0
:101128009FEBFAC8D93120120377665445BDAC9EAF
:101138008FFBEAD8C94253617004152736CEDFED1C
:10114800FC8899ABBA5243716014053726DECFFD8F
:10115800EC9889BBAA6372405125340617EFFECC80
:10116800DDA9B88A9B7362504135241607FFEEDC6F
:10117800CDB9A89A8B8495A7B6C2D3E1F008192BEC
:101188003A4E5F6D7C9485B7A6D2C3F1E018093B4F
:101198002A5E4F7D6CA5B48697E3F2C0D129380A40
:1011A8001B6F7E4C5DB5A49687F3E2D0C139281A2F
:1011B8000B7F6E5C4DC6D7E5F48091A3B24A5B699C
:1011C800780C1D2F3ED6C7F5E49081B3A25A4B790F
:1011D800681C0D3F2EE7F6C4D5A1B082936B7A4800
:1011E800592D3C0E1FF7E6D4C5B1A092837B6A58EF
:1011F800493D2C1E0F0089129B24AD36BF48C15AA9
:10120800D36CE57EF78108931AA52CB73EC940DB5D
:1012180052ED64FF76028B109926AF34BD4AC3584D
:10122800D16EE77CF5830A9118A72EB53CCB42D93D
:1012380050EF66FD74048D169F20A932BB4CC55E25
:10124800D768E17AF3850C971EA128B33ACD44DF1D
:1012580056E960FB72068F149D22AB30B94EC75C0D
:10126800D56AE378F1870E951CA32AB138CF46DDFD
:1012780054EB62F97008811A932CA53EB740C95205
:10128800DB64ED76FF89009B12AD24BF36C148D3DD
:101298005AE56CF77E0A8318912EA73CB542CB50CD
:1012A800D966EF74FD8B029910AF26BD34C34AD1BD
:1012B80058E76EF57C0C851E9728A13AB344CD56A5
:1012C800DF60E972FB8D049F16A920BB32C54CD79D
:1012D8005EE168F37A0E871C952AA338B146CF548D
:1012E800DD62EB70F98F069D14AB22B930C74ED57D
:0512F8005CE36AF178DF
:103CB10052668D00000000000000000000000000BE
:053CC1000000000000FE
:013D6100223F
:03002300022BD3DA
:102BD300C0E0C083C082C0D075D0183098677551EB
:102BE30001AF9920020CEF64027058750905D202F7
:102BF3008051300F14C20FAE0E050E74AE2EF58247
:102C0300E43467F583EFF08037BF0904D20F8030D7
:102C1300BF0205530E808028BF03159067ACE50EF5
:102C2300F0630E80530E80C202D208750900801033
:102C3300AE0E050E74AE2EF582E43467F583EFF025
:102C4300750905C29830996E3003693010073097C3
:102C530004D200805F9066A1E0FFE510C39F400FA0
:102C6300C203D213200B02D215C20BD2968045AFFA
:102C730010051074AE2FF582E43468F583E0F51186
:102C830030091953117F30012820D0082004226312
:102C93001180801D30041A6311808015300112E504
:102CA300115211300406A2D0929B8005A2D0B39298
:102CB3009B851199C299D2AFD0D0D082D083D0E076
:012CC30032DE
:1038FD008F2F9067ADE0FF04F074A22FF582E434B2
:10390D0066F5837420F0E4FFEFC39D503BE52F7502
:10391D00F003A424D0F582E43410F583E493FB7412
:10392D000193FA740293F98F82758300121AB8FE0F
:10393D009067ADE024A2F582E43466F583EEF00FD6
:09394D009067ADE004F080C02297
:103BFF00742D2FF582E43461F583E0FE64206016A6
:103C0F009067ADE0FD04F074A22DF582E43466F503
:073C1F0083EEF00F80DA22B2
:101D1000C209C204C201C212C210D20CE4F50AD236
:101D2000139069AE74FFF0A374B8F0C20AC205C282
:101D300011E4F50DF50FF527E52775F003A424D080
:101D4000F582E43410F583E493FB740193FA740292
:101D500093F9121A9F7003021F69E4F529F52AF519
:101D600028742D2528F582E43461F583E0FF7003A3
:101D7000021F64E52775F003A424D0F582E4341033
:101D8000F583E493FB740193FA740293F985298235
:101D9000758300121AB8FEEFB50608752A010529E9
:101DA000021F5FE52A7003021F5FEE6003021F5AE5
:101DB000AD29AF271238FDE527B40E004003021FFE
:101DC00064901DC8F8282873021DF2021E3E021EF0
:101DD00043021E48021E7A021EB3021EB3021EB345
:101DE000021EE4021EEA021EEE021EF4021EFA02A7
:101DF0001F2AAF28123BFF742D2528F9E43461FA1D
:101E00007B01C0031B8B32753300753400E4F5355C
:101E1000D0031221538F2E8E2D8D2C8C2BAB2EAAFE
:101E20002DA92CA82B7F007E8C7D0A7C00121B33F1
:101E3000121BC59069AEEEF0A3EFF0021F64C20C56
:101E4000021F64D210021F64AF28123BFF742D25BD
:101E500028F9E43461FA7B01C0031B8B327533002F
:101E6000753400E4F535D0031221538F2E8E2D8D5D
:101E70002C8C2BAF2E8F0A021F64AF28123BFF74ED
:101E80002D2528F582E43461F583E0B43702D209C8
:101E9000742E2528F582E43461F583E0FFB44E0406
:101EA000C2018002D201EF64456003021F64D204C4
:101EB000021F64AF28123BFF742D2528F9E434611A
:101EC000FA7B01C0031B8B32753300753400E4F5D7
:101ED00035D0031221538F2E8E2D8D2C8C2B852ED9
:101EE00008021F64D201D204807AD2018076D20522
:101EF000D2118070D205D20A806AAF28123BFF74DB
:101F00002D2528F9E43461FA7B01C0031B8B32755F
:101F10003300753400E4F535D0031221538F2E8E33
:101F20002D8D2C8C2B852E0F803AAF28123BFF7401
:101F30002D2528F9E43461FA7B01C0031B8B32752F
:101F40003300753400E4F535D0031221538F2E8E03
:101F50002D8D2C8C2B852E0D800AE4F52AF5290574
:0A1F600028021D610527021D38222A
:103252007BFF7A0E79751217A59069AEE0FEA3E0A6
:10326200FFC3E49FFFE49EFEAB07FA3395E0F9F853
:103272007F007E8C7D0A7C00121B338F328E318D53
:10328200308C2F7BFF7A0E79B11217A57BFF7A0F54
:103292007909A210E433F52F1217A57BFF7A0F7973
:1032A2003F850A2F1217A57BFF7A0F796BA209E4DB
:1032B20033F52F1217A57BFF7A0F798CA201E43325
:1032C200F52F1217A57BFF7A0F79B5A204E433F527
:1032D2002F1217A57BFF7A0F79DCA211E433F52FA9
:1032E2001217A57BFF7A107907A20AE433F52F1291
:0332F20017A522FB
:102AD7007E107F351235BBEF4E70037F01227E10CB
:102AE7007F381235BBEF4E60231238A0A804A90522
:102AF700AA06AB077F007E8C7D0A7C00121B33126F
:102B07001BC59069AEEEF0A3EFF0800A9069AE7432
:102B1700FFF0A374B8F07E107F3E1235BBEF4E6016
:102B27000C123CC7EF24D024FF92108002C2107E03
:102B3700107F441235BBEF4E60071238A08F0A8012
:102B470003E4F50A7E107F4A1235BBEF4E600C1284
:102B57003CC7EF24D024FF92098002C2097E107F70
:102B6700501235BBEF4E600C123CC7EF24D024FF48
:102B770092018002C2017E107F561235BBEF4E6074
:102B87000C123CC7EF24D024FF92048002C2047EBB
:102B9700107F5C1235BBEF4E600E123CC7EF24D09E
:102BA70024FF920592118004C205C2117E107F6333
:102BB7001235BBEF4E600E123CC7EF24D024FF92B4
:0C2BC70005920A8004C205C20A7F0022A9
:1030EE00C203C215C208C202C20FE4F5109066A157
:1030FE00F0F50EF551C200D297D296750CFF90677F
:10310E00ADF075080CC206C21490669F7409F0A348
:10311E00F0750F05C209C204C201C212C210D20C50
:10312E00E4F50AF509D2139069AE74FFF0A374B8F2
:10313E00F0C20AC205C211E4F50D122AD7EF6003E0
:10314E00121D10E49067A2F0C2ADF5C9D2CDD2CC5B
:10315E00C2C9C2CAF5CDF5CC9069AEE0F5CBA3E0FD
:10316E00F5CA85CBCD85CACCE4F59830010C200983
:10317E00095387BFD29FD29E8002D29E438740C200
:10318E009FC2ACC298C29975B81075B710D2CAD288
:04319E009CD2AC22F1
:103CE100E5136FFF9011FD936512F513EF9010FD31
:043CF10093F5122213
:013D6200223E
:102778008E288F29E4F52AF513F512AA06A9077BF6
:10278800018B2E8A2F89309067A2E0121AE5740116
:102798002530F530E4352FF52F30050F9067A3E08D
:1027A800AB2EAA2FA930121AE5800D9066A0E0ABD7
:1027B8002EAA2FA930121AE5752E0185282F8529F2
:1027C800300D0DE4FEEEC39D5018AB2E0530E530FC
:1027D800AA2F7002052F14F9121A9FFF123CE10E5E
:1027E80080E3AB2E0530E530AA2F7002052F14F9CF
:1027F800E513121AE5AB2EAA2FA930E512121AE535
:102808000D0D752C68752DAE752E0185282F85291F
:1028180030852D82852C837402F0052DE52D7002FC
:10282800052C052AE4FEEEC39D504EAB2EAA2FA917
:1028380030121A9FF52B6402600BE52B64036005C8
:10284800E52BB40913852D82852C837409F0052D99
:10285800E52D7002052C052A852D82852C83E52B14
:10286800F0052DE52D7002052C052A74012530F59B
:1028780030E4352FF52F0E80AD852D82852C83749D
:1028880003F0052DE52D7002052C052A906693E0CE
:10289800FCA3E0FDA3E0FEA3E0FFE4FAF9F8EF24CF
:1028A80001FFEA3EFEE93DFDE83CFC906693121B01
:1028B800E430240D7E107F6A7C687DAEAB2A122836
:0428C800CCAF2A2245
:10303200E4FF9066A0E0FE7D000FED2405F582E43A
:103042003461F583EEF00F74052401F582E43461F6
:10305200F583E4F07C667D92FEED1DAA0470011CEE
:10306200F5828A83E0FBAA070F74052AF582E4340D
:1030720061F583EBF00EBE04E07C667D96E4FEED26
:103082001DAA0470011CF5828A83E0FBAA070F7453
:10309200052AF582E43461F583EBF00EBE04E07C90
:1030A200667D9AE4FEED1DAA0470011CF5828A83F6
:1030B200E0FBAA070F74052AF582E43461F583EB7D
:1030C200F00EBE04E07C667D9EE4FEED1DAA047057
:1030D200011CF5828A83E0FBAA070F74052AF58298
:0C30E200E43461F583EBF00EBE04E02244
:083D5200C2992099FDD29922CB
:093D4900D2CAD29CD2ACC20822FD
:103B1600AD077E677FA21227789066A1EFF0D203E9
:103B2600E4F51030240D7E107F797C687DAEE0FBD5
:103B36001228CCC296301003D20022E50A6003F5A3
:063B46004E22123D522246
:1039AF008F2730030F30244E7E107F85E4FBFDFC04
:1039BF001228CC22906378E09066A0F0300C117E34
:1039CF00637F77E52724FCFD1227789066A1EFF03F
:1039DF00A21182055005750B05D214E4F510D20320
:1039EF00C296301004D200800BE50A6004F54E80B9
:0739FF0003123D52C2152224
:1022F700200603300B037F0022200803022480C23C
:1023070008E4906475F09067ACE0FF547F24FCF517
:1023170027906476F090667AE0906477F0EF5480C7
:10232700FF24AFF582E43467F583E0906478F074B6
:10233700AE2FF582E43467AD82FCE4F513F512FEA7
:102347009067ACE0547FF9EEC39950140DEDAA04E1
:1023570070010C14F5828A83E0FF123CE10E80E0E5
:10236700E512451360443024197E107F939067ACC3
:10237700E0548024AEF582E43467AD82FCAB0112F1
:1023870028CC906697E0FCA3E0FDA3E0FEA3E0FF66
:10239700E4FAF9F8EF2401FFEA3EFEE93DFDE83CE7
:1023A700FC906697121BE40224803005249067ACEA
:1023B700E05480FF24AEF582E43467F583E090674C
:1023C700A2F074AF2FF582E43467F583E09067A33A
:1023D700F0E5277039C214F50B9067A3E0B4E01E4F
:1023E7007490F0200503022480D2062024030224DF
:1023F700807E107FA2E4FBFDFC1228CC807B30247A
:10240700787E107FB8E4FBFDFC1228CC806B9067C8
:10241700ACE0548024B0F582E43467F58363A2010D
:1024270090647963A201AF2712204530241C7E10E7
:102437007FC19067ACE0FB548024AEF582E434673B
:10244700AD82FCEB547FFB1228CC90668FE0FCA397
:10245700E0FDA3E0FEA3E0FFE4FAF9F8EF2401FFB3
:10246700EA3EFEE93DFDE83CFC90668F121BE4A2C4
:102477000A82055002D206D216301605C2167F010F
:04248700227F00228E
:05001E00C2AEC2AC22DD
:103A0600300008209705C200123D52E54EB401066B
:103A1600E4F54E123D52302523C225E509600BD54B
:103A26000908630E80530E80C20230110FE50B6049
:103A36000BD50B08E4F510D203750B05A20A820616
:0F3A4600500C200309E4FF123B16C206D20B22DC
:0E3D1400301508201405C2157F01227F002201
:103956009080007480F090633663A201F583F5824F
:1039660063A2017F0812204590633E63A201908006
:103976008863A2017F0A122045908092E4F0A37426
:1039860032F0A37401F0906348E0FF9080B1F090AC
:1039960080E1EFF09080957455F0A3F0908000746C
:0939A60001F090800974F0F02298
:10374900908009E04410F09080A0E0706C9080A116
:103759007482F09080A874FFF0A3F0A3F0A3F07F27
:10376900039080AEEFF07FCBA3EFF07F039080ACA6
:10377900EFF0A374CBF09080007402F09069B4125A
:103789001BF0000000009069B4E0908040F090695F
:10379900B5E0908041F09069B6E0908042F0906980
:1037A900B7E0908043F0A3E4F0A3F0A3F0A3F09076
:0A37B9008018F0A3F0A3F0A3F022A3
:10383D00908009E04440F09080D17482F09063490B
:10384D00E0FF9080DEF090634AE0FF9080DFF09023
:10385D0080027402F09069B8121BF0000000009015
:10386D0069B8E0908058F09069B9E0908059F09077
:10387D0069BAE090805AF09069BBE090805BF0A34C
:10388D00E4F0A3F0A3F0A3F0908030F0A3F0A3F048
:03389D00A3F02273
:1037C300908009E04420F09080B8E0706C9080B95C
:1037D3007482F07F039080C6EFF07FCDA3EFF07F7C
:1037E300039080C4EFF0A374CDF09080C074FFF019
:1037F300A3F0A3F0A3F09080017402F09069BC12CF
:103803001BF0000000009069BCE090804CF09069D0
:10381300BDE090804DF09069BEE090804EF09069DD
:10382300BFE090804FF0A3E4F0A3F0A3F0A3F090E7
:0A3833008024F0A3F0A3F0A3F0221C
:1036C5008C278D28A907EAFDE975F018A424ACFF1D
:1036D500E5F034808F82F583EDF0EBFDE975F018A8
:1036E500A4FFAEF024ACFBEE34808B82F583A3ED12
:1036F500F08528828C83E0FDEF24A8FFEE3480FE60
:103705008F82F583EDF08528828C83A3E08F828EEE
:1037150083A3F0852882852783A3A3E0FDE975F0BF
:1037250018A424A8FFE5F03480FE8F82F583A3A3B7
:10373500EDF08528828C83A3A3A3E08F828E83A3DB
:04374500A3A3F02228
:1034AD008D2CAB07AA06908000E030E5079065787B
:1034BD007401F0229069B4E0FCA3E0FDA3E0FEA34B
:1034CD00E0F5308E2F8D2E8C2DAE02AF038E838FB7
:1034DD008263A201E52F540744C0F58385308263D2
:1034ED00A201AF2C1220B7E4FCFDFEE530252CF532
:1034FD0030EE352FF52FED352EF52EEC352DF52D36
:10350D00908040E52DF0A3E52EF0A3E52FF0A3E587
:10351D0030F09080007420F0AF30AE2FAD2EAC2D7A
:07352D009069B4121BE422B7
:103534008D27AB07AA06908002E030E507906578F6
:103544007403F0229069B8E0FCA3E0FDA3E0FEA3BD
:10355400E0F52B8E2A8D298C28AE02AF038E838F43
:103564008263A201E52A540744D0F583852B826344
:10357400A201AF271220B7E4FCFDFEE52B2527F5B9
:103584002BEE352AF52AED3529F529EC3528F528D1
:10359400908058E528F0A3E529F0A3E52AF0A3E5F7
:1035A4002BF09080027420F0AF2BAE2AAD29AC280A
:0735B4009069B8121BE4222C
:1031A2008F27908001E030E5099065787402F07F06
:1031B20000229069BCE0FCA3E0FDA3E0FEA3E0F5E1
:1031C2002B8E2A8D298C2890667B63A201E52A54D6
:1031D2000744C8F583852B8263A2017F061220CDA6
:1031E200E52B2406F52BE4352AF52AE43529F529C1
:1031F200E43528F52890657963A201E52A5407444D
:10320200C8F583852B8263A201AF271220CDE4FC8F
:10321200FDFEE52B2527F52BEE352AF52AED35297E
:10322200F529EC3528F52890804CE528F0A3E5290E
:10323200F0A3E52AF0A3E52BF09080017420F0AF13
:103242002BAE2AAD29AC289069BC121BE4AF272211
:1029D3009081E0E0F527052705270527052705272B
:1029E30005270527052705270527908010E0F52AE9
:1029F300A3E0F52BA3E0F52CA3E0F52D9081E1E016
:102A0300F527052705270527052705270527052773
:102A1300052705270527908014E0F52EA3E0F52F61
:102A2300A3E0F530A3E0F531E530B52C08E531B589
:102A33002D037F0022E4F527E530540744E0F583B6
:102A430085318263A20190637563A2017F0812201E
:102A5300FD90637763A2019062AE63A2017F0612C9
:102A63002045906375E0F528A3E0F529E4F5279068
:102A73006375E0702AA3E024F8F527E53054074492
:102A8300E0F58385318274082582F582E43583F588
:102A93008363A20190637563A201AF271220FDAE89
:102AA30028E4FCFDE5312529F531E5303EF530ED2F
:102AB300352FF52FEC352EF52E908014E52EF0A34F
:102AC300E52FF0A3E530F0A3E531F09080007440EA
:042AD300F0AF272217
:10248B009081E6E0F5270527052705270527052772
:10249B0005270527052705270527908028E0F52A1E
:1024AB00A3E0F52BA3E0F52CA3E0F52D9081E7E05D
:1024BB00F5270527052705270527052705270527C1
:1024CB0005270527052790802CE0F52EA3E0F52F97
:1024DB00A3E0F530A3E0F531E4F527E530B52C0AA0
:1024EB00E531B52D05C21F0225F7E530540744F041
:1024FB00F58385318263A20190637563A2017F0826
:10250B001220FD906375E0F528A3E0F529E5294538
:10251B002870099080027410F07F0022906682E090
:10252B00FFF46030906377E06F60030225BE906626
:10253B0083E0FF906378E06F7079906684E0FF90A2
:10254B006379E06F706D906685E0FF90637AE06F62
:10255B006031805F906377E0906682F0906378E003
:10256B00906683F0906379E0906684F090637AE0F4
:10257B00906685F090637BE0FFA3E0906349CFF01A
:10258B00A3EFF0906375E0702AA3E024F8F527E53C
:10259B0030540744F0F58385318274082582F58227
:1025AB00E43583F58363A20190637563A201AF27C2
:1025BB001220FDAE28E4FCFDE5312529F531E5308F
:1025CB003EF530ED352FF52FEC352EF52EAF2DAE2C
:1025DB002CAD2BAC2AAB31AA30A92FA82ED3121BB2
:1025EB00D340099080027410F07F002290802CE57C
:1025FB002EF0A3E52FF0A3E530F0A3E531F09080AA
:07260B00027440F0AF27222A
:102612009081E3E0F52705270527052705270527EC
:102622000527052705270527052790801CE0F52AA1
:10263200A3E0F52BA3E0F52CA3E0F52D9081E4E0D7
:10264200F527052705270527052705270527052738
:10265200052705270527908020E0F52EA3E0F52F1A
:10266200A3E0F530A3E0F531E4F527E530B52C0A17
:10267200E531B52D05C22002275DE530540744E857
:10268200F58385318263A20190600463A2017F0E0B
:10269200122113906004E0F528A3E0F52990600C64
:1026A200E0FFF4604590667BE0FEEF6E706EA3E0A3
:1026B200FF90600DE06F706490667DE0FF90600EA9
:1026C200E06F705890667EE0FF90600FE06F704C94
:1026D20090667FE0FF906010E06F7040906680E04F
:1026E200FF906011E06F60048032D2D9906004E004
:1026F200702AA3E024F2F527E530540744E8F58375
:10270200853182740E2582F582E43583F58363A2D6
:102712000190600463A201AF27122113AE28E4FCEA
:10272200FDE5312529F531E5303EF530ED352FF562
:102732002FEC352EF52EAF2DAE2CAD2BAC2AAB31B6
:10274200AA30A92FA82ED3121BD35006E52945285B
:1027520070099080017410F07F0022908020E52E95
:10276200F0A3E52FF0A3E530F0A3E531F09080016E
:062772007440F0AF2722C5
:102CC4008E2C8F2D908000E030E50790657874019C
:102CD400F0229069B4E0FCA3E0FDA3E0FEA3E0F5DC
:102CE400338E328D318C30E533FFE5325407FEE408
:102CF4002FF52FEE34C0F52E852F82F5837423F043
:102D0400052FE52F7002052E532EC7F582852E83DD
:102D1400740AF0052FE52F7002052E532EC7906319
:102D24003E63A201852E83852F8263A2017F061252
:102D340020B77406252FF52FE4352EF52E852C8328
:102D4400852D8263A201852E83852F8263A20112C1
:102D5400209BE4FCFDFE9069B4E0F8A3E0F9A3E055
:102D6400FAA3E02FFFEE3AFEED39FDEC38FCEF2438
:102D740008FFE43EFEE43DFDE43CFC9069B4121B14
:102D8400E49069B4E0908040F09069B5E0908041AF
:102D9400F09069B6E0908042F09069B7E09080438B
:082DA400F09080007420F02281
:1028CC008E318F328C338D348B35908000E030E537
:1028DC00079065787401F0229069B4E0FCA3E0FDE8
:1028EC00A3E0FEA3E0F53B8E3A8D398C38E53BFF37
:1028FC00E53A5407FEE42FF537EE34C0F53685374C
:10290C0082F5837423F00537E537700205365336AC
:10291C00C7F582853683740AF00537E537700205F2
:10292C00365336C790633E63A20185368385378262
:10293C0063A2017F061220B774062537F537E435FC
:10294C0036F53685318385328263A20185368385DF
:10295C00378263A20112209B8F3CEF2537F537E4B9
:10296C003536F536E535601785338385348263A2B9
:10297C000185368385378263A201AF351220B7E516
:10298C003C24082535F535FFE4FCFDFEE53B2FF531
:10299C003BEE353AF53AED3539F539EC3538F53855
:1029AC00908040E538F0A3E539F0A3E53AF0A3E5D3
:1029BC003BF09080007420F0AF3BAE3AAD39AC38B0
:0729CC009069B4121BE42224
:102E8D008E458F468D47908000E030E50790657840
:102E9D007401F0229069B4E0FCA3E0FDA3E0FEA371
:102EAD00E0F54D8E4C8D4B8C4AE54DFFE54C5407AE
:102EBD00FEE42FF549EE34C0F548854982F583745B
:102ECD0023F00549E549700205485348C7F5828549
:102EDD004883EBF00549E549700205485348C79012
:102EED00633E63A20185488385498263A2017F0603
:102EFD001220B774062549F549E43548F54885454E
:102F0D008385468263A20185488385498263A20138
:102F1D00AF471220B774082547F547FFE4FCFDFEC7
:102F2D00E54D2FF54DEE354CF54CED354BF54BECA8
:102F3D00354AF54A908040E54AF0A3E54BF0A3E50C
:102F4D004CF0A3E54DF09080007420F0AF4DAE4CE9
:0B2F5D00AD4BAC4A9069B4121BE4229B
:103640008F40908000E030E5079065787401F022AB
:103650009069B4E0FCA3E0FDA3E0FEA3E0F5448E96
:10366000438D428C41E544FFE5435407FEE42FFFC0
:10367000EE34C09062B463A201F5838F8263A2012D
:10368000AF401220B7E4FCFDFEE5442540F544EED2
:103690003543F543ED3542F542EC3541F541908037
:1036A00040E541F0A3E542F0A3E543F0A3E544F093
:1036B0009080007420F0AF44AE43AD42AC419069BD
:0536C000B4121BE4221E
:102DAC008E278F28AB05908000E030E50790657882
:102DBC007401F0229069B4E0FCA3E0FDA3E0FEA353
:102DCC00E0F52E8E2D8D2C8C2BE52EFFE52D54074A
:102DDC00FEE42FF52AEE34C0F529852A82F583749A
:102DEC0023F0052AE52A700205295329C7F58285A7
:102DFC002983EBF0052AE52A7002052990633E63CE
:102E0C00A201852983852A8263A2017F061220B73D
:102E1C007406252AF52AE43529F5295329C7E5270F
:102E2C00852A82852983F0052AE52A700205295313
:102E3C0029C7F582852983E528F0052AE52A700241
:102E4C0005295329C7E52E240AF52EE4352DF52D39
:102E5C00E4352CF52CE4352BF52B908040E52BF04C
:102E6C00A3E52CF0A3E52DF0A3E52EF090800074E3
:102E7C0020F0AF2EAE2DAD2CAC2B9069B4121BE410
:012E8C002223
:1032F500E4F527E5272401FFE433FE123A9C7436F2
:103305002527F582E43463F583EFF00527E527C328
:10331500943F40DFE4F527E527247FFFE433FE12E1
:103325003A9C742D2527F582E43461F583EFF0741A
:103335002D2527F582E43461F583E0FF6003B4FFB2
:103345001D742D2527F582E43461F5837420F0740E
:103355002E2527F582E43461F583E4F080090527FD
:10336500E527C3948040B0E49061ACF0F527AF2722
:103375007E00123A9C74AD2527F582E43461F5830D
:0C338500EFF00527E527C394FE40E3228B
:103C6E00E4FDFCC3ED9FEC9E5015E4FBFA0BBB008C
:103C7E00010ABA01F8BB90F50DBD00010C80E422DB
:0D3D22004390014390025390FE5390FD2208
:0D3D2F005390FD5390FE43900243900122FB
:0F3D05005390FD439002E5905408FF5390FD2228
:0D3D3C005390FD4390014390025390FD22EF
:073D5A00AE071FEE70FA2214
:103B8000AD07E4FC5390FDEDA804088002C333D8D0
:103B9000FC30E70543900180035390FE7F05123D02
:0C3BA0005A4390020CBC08DC5390FD223C
:103BD600E4FF5390FD7E07439002E59030E00D74BC
:103BE60001A806088002C333D8FC42075390FD1E85
:093BF600C3EE6480948050DF22CC
:103BAC00AB05AA07123D227FA0123B80123D05AF48
:103BBC0002123B80123D05AF03123B80123D0512F1
:0A3BCC003D2F7F0A7E00123C6E229E
:103A9C00AB07AA06C3EB94FFEA9400400DE42BF5A8
:103AAC008274773AF583E493FF22123D227FA012B1
:103ABC003B80123D05AF03123B80123D05123D22A7
:103ACC007FA1123B80123D05123BD6123D3C123DAC
:023ADC002F2297
:103B4C008B2CA2AF9227C2AF85A22D53A2FE8E83DF
:103B5C008F8205A28C838D827409122141E52C532E
:103B6C00A2FE43A22012214353A2DF852DA2A2273D
:043B7C0092AFFF22E3
:103C8E00A2AF9227C2AF8C838D82EF12214143A245
:0D3C9E002012214353A2DFA22792AFFF2284
:103C26008F27A2AF9227C2AFE4F5838D8274061266
:103C36002141E52743A22012214353A2DFA2279266
:043C4600AF7F012229
:103C4A008F27A2AF9227C2AFE4F5838D82740A123E
:103C5A002141E52743A22012214353A2DFA2279242
:043C6A00AF7F012205
:101F6A00A907E7FFA805EF93C3966008403B74FCF6
:101F7A002FFF80F00F08EF93C3966008402B74FB85
:101F8A002FFF80E00F08EF93C3966008401B74FA96
:101F9A002FFF80D00F08EF93D3966008400B74F997
:101FAA002FFF80C01F1F1F1F1FEF54FEF80303F7E8
:101FBA00E893FC08E893FD08E893FE08E893FF22FB
:101FCA0009E993C39D6008402974FB29F980F10946
:101FDA00E993C39E6008401A74FA29F980E209E974
:101FEA0093D39F6008400B74F929F980D319191902
:101FFA001919E9C313C313FF22740093F8ECC398A9
:10200A004024701F740193F8EDC39840197014743A
:10201A000293F8EEC398400E7009740393F8EFC365
:10202A009840037F00227F0122EDF8E6F008A3DF43
:10203A00FA22EDF8E0F608A3DFFA22E0A363A20190
:10204A00F0A363A201DFF475A2002263A201F0A348
:10205A0063A20122E0A363A201F0A363A201E0A3A9
:10206A0063A201F0A363A201E463A201F0A363A245
:10207A0001DFE175A20022E0A363A2016DFE936C69
:10208A00FDEE058393FC158363A201DFEA75A200C6
:10209A00227F00E493A363A201F00F600CA3E583FF
:1020AA00C2E3F58363A20180EA75A20022E0A3637A
:1020BA00A201F0A3E583C2E3F58363A201DFEE7513
:1020CA00A20022E0A363A201F0A3E583C2E4D2E363
:1020DA00F58363A201DFEC75A20022E0A363A201EB
:1020EA00F0A3E58344F8C2E5F58363A201DFEC754A
:1020FA00A20022E583C2E3F583E0A363A201F0A371
:10210A0063A201DFEE75A20022E583C2E4D2E3F501
:10211A0083E0A363A201F0A363A201DFEC75A2002E
:10212A0022E58344F8F583E0A363A201F0A363A246
:10213A0001DFEE75A20022F922C002C004C0061215
:09214A00FFF0D006D004D00222FF
:10342D0002084FE493A3F8E493A34003F68001F25E
:10343D0008DFF48029E493A3F85407240CC8C333A0
:10344D00C4540F4420C8834004F456800146F6DF6F
:10345D00E4800B0102040810204080903CABE47E18
:10346D00019360BCA3FF543F30E509541FFEE49364
:10347D00A360010ECF54C025E060A840B8E493A32B
:10348D00FAE493A3F8E493A3C8C582C8CAC583CA56
:10349D00F0A3C8C582C8CAC583CADFE9DEE780BE0E
:013CC60000FD
:101A9F00BB010689828A83E0225002E722BBFE0245
:091AAF00E32289828A83E4932278
:101AB800BB010CE58229F582E5833AF583E02250E3
:101AC80006E92582F8E622BBFE06E92582F8E2222D
:0D1AD800E58229F582E5833AF583E4932247
:101AE500BB010689828A83F0225002F722BBFE01E0
:021AF500F322DA
:101AF70075F008758200EF2FFFEE33FECD33CDCCA6
:101B070033CCC58233C5829BED9AEC99E582984028
:101B17000CF582EE9BFEED9AFDEC99FC0FD5F0D605
:101B2700E4CEFBE4CDFAE4CCF9A88222B800C1B92F
:101B37000059BA002DEC8BF084CFCECDFCE5F0CB6D
:101B4700F97818EF2FFFEE33FEED33FDEC33FCEBA6
:101B570033FB10D703994004EB99FB0FD8E5E4F961
:101B6700FA227818EF2FFFEE33FEED33FDEC33FC4E
:101B7700C933C910D7059BE99A4007EC9BFCE99A42
:101B8700F90FD8E0E4C9FAE4CCFB2275F010EF2F87
:101B9700FFEE33FEED33FDCC33CCC833C810D70787
:101BA7009BEC9AE899400AED9BFDEC9AFCE899F8C2
:0E1BB7000FD5F0DAE4CDFBE4CCFAE4C8F92255
:0E1BC500C3E49FFFE49EFEE49DFDE49CFC2231
:101BD300EB9FF5F0EA9E42F0E99D42F0E89C45F068
:011BE30022DF
:0C1BE400ECF0A3EDF0A3EEF0A3EFF02274
:101BF000A8828583F0D083D082121C07121C0712A2
:101C00001C07121C07E473E493A3C583C5F0C583C6
:101C1000C8C582C8F0A3C583C5F0C583C8C582C83E
:011C200022A1
:10174300E53B242FF8E6053B22782C302E02782F38
:10175300E475F001121C70021A9F2027EB7F2ED232
:10176300278018EF540F2490D43440D4FF302B0B30
:10177300EF24BFB41A0050032461FFE53C60021557
:101783003C053FE53F7002053E302E0D782CE47595
:10179300F001121C70EF021AE5023A557403D22EBF
:1017A3008003E4C22EF53B8B2C8A2D892EE4F53C75
:1017B300F53EF53FE53C60077F2012177E80F57507
:1017C3003DFFC228C227C229C22AC22CC22DC22F62
:1017D30012174CFF700D302E057F0012178FAF3F8D
:1017E300AE3E22B4255FC2D5C22B12174CFF24D0C4
:1017F300B40A00501A75F00A783C30D50508B6FFD4
:101803000106C6A426F620D5047002D22A80D92464
:10181300CFB41A00EF5004C2E5D22B02198FD2289D
:1018230080C6D22780C0D22980BCD2D580BAD22C20
:1018330080B47F2012177E2029077401B53C004035
:10184300F1121743FF12177E0217B7D22FD22D8042
:1018530095121743FB121743FA121743F94A4B70B9
:101863000679607A1A7BFF20292EE53C602A7E00E8
:101873008E82758300121AB860060EEE653D70F015
:10188300C2D5EBC0E0EAC0E0E9C0E0EE1219D6D061
:10189300E0F9D0E0FAD0E0FB121A9FFF60AAEBC098
:1018A300E0EAC0E0E9C0E012177ED0E02401F9D0FD
:1018B300E03400FAD0E0FBE53D0460DCD53DD9809F
:1018C300877BFF7A1979D2D229809C79108002799B
:1018D30008C22DC22F8008D2D5790A8004790AC2A2
:1018E300D5E53D047002F53DE4FAFDFEFF12174312
:1018F300FC7B08202813121743FD7B1030270A12A4
:101903001743FE121743FF7B20EC3382D592D55049
:1019130013C3E43027069FFFE49EFEE42028039DC3
:10192300FDE49CFCE4CBF8C228EC700CCFCECDCC0C
:10193300E824F8F870F38017C3EF33FFEE33FEEDBE
:1019430033FDEC33FCEB33FB994002FB0FD8E9EB9F
:10195300302805F8D0E0C448B228C0E00AEC4D4E68
:101963004F78207B0070C2EAB53D0040BCC0E01256
:1019730019D8D0F0D0E0202804C4C0E0C4B228C0F5
:10198300F0121767D0F0D5F0EB0217B7121CCF187F
:10199300545318CE5818254C18214218D24F18DA30
:0F19A3004418DA49183A4318E05518C44618C4D6
:1019B2004518C4471A805018292D182D2E18502B5F
:1019C200183123184E201A692A17E94800001848CE
:1019D2003F3F3F00790AA2D5202A14302C09B910C2
:1019E200020404B9080104A2D5202D0250010420EA
:1019F20029689229B53C005034C0E07F20302A1972
:101A02007F30A229722D722C500F121A2FC229C2B6
:101A12002DC22CC22F7F30800F302C03E9C0E01280
:101A2200177E302C03D0E0F9D0E0B53CCC302C1737
:101A32007F30B9100C12177E7F58302B077F7880C9
:101A420003B9080312177E3029057F2D02177E7F06
:101A520020202FF87F2B202DF322922980CF286E71
:101A6200756C6C2900D2281217433028F8C22878E6
:101A72003C30D50108F60217E92D50434958121798
:101A8200432403B405004001E4901A7B9312176FBC
:0D1A9200743A12176FD22A753C040218CE68
:102153008B2F8A308931E4F53BF53AF539F538F5BB
:1021630036F537E533453445326012EBC0E0EAC05B
:10217300E0E9C0E0AB32AA33A934121C80AB2F05CF
:1021830031E531AA307002053014F9121A9FF53C7B
:10219300C394094007E53CD3940D40E1E53C64203A
:1021A30060DBE53CB42D054337038016E53CB42BD7
:1021B30005433701800C74FF2531F53174FF353049
:1021C300F530E53560046410703FAB2FAA30A931B8
:1021D300121A9F64306009E535702E75350A80291F
:1021E300900001121AB8FF64786004EFB4581343E7
:1021F300370175351074022531F531E43530F5308A
:102203008007E5357003753508AB2F0531E531AA35
:10221300307002053014F9121A9FF53CC3946140E3
:102223000AE53CD3947A5003533CDF74D0253CF544
:102233003CC3940A400CE53C9411406D74F9253C71
:10224300F53CE53CD395355060433701853B4085EC
:102253003A3F85393E85383DAF357E00E4FCFDAB22
:102263003BAA3AA939A838121C21C8ECC8C9EDC940
:10227300CAEECACBEFCBE4FCFDFEEB253CF53BEE0F
:102283003AF53AED39F539EC38F538AF3BAE3AADBE
:1022930039FCAB40AA3FA93EA83DD3121BD3500340
:1022A30002220C43370402220CE53720E003E480CA
:1022B3002DE53345344532601EAB2FE53124FFF95C
:1022C300E53034FFFAEBC0E0EAC0E0E9C0E0AB324E
:1022D300AA33A934121C80E53730E20774FFFFFEEE
:1022E300FDFC22E537AF3BAE3AAD39AC3830E10304
:0422F300021BC522E3
:101C2100E88FF0A4CC8BF0A42CFCE98EF0A42CFC62
:101C31008AF0EDA42CFCEA8EF0A4CDA8F08BF0A4E0
:101C41002DCC3825F0FDE98FF0A42CCD35F0FCEB3F
:101C51008EF0A4FEA9F0EB8FF0A4CFC5F02ECD3904
:0F1C6100FEE43CFCEAA42DCE35F0FDE43CFC2271
:101C7000FAE6FB0808E6F925F0F618E6CA3AF62275
:101C8000BB011A89828A83D0F0D0E0F8D0E0F9D085
:101C9000E0FAD0E0FBE8C0E0C0F0021CFE5016E91C
:101CA000F8D083D082D0E0F9D0E0FAD0E0FBC08257
:101CB000C083021CF5BBFE16E9F8D083D082D0E0C9
:0F1CC000F9D0E0FAD0E0FBC082C083021D0722FA
:101CCF00D083D082F8E4937012740193700DA3A3A4
:101CDF0093F8740193F5828883E4737402936860B8
:061CEF00EFA3A3A380DFB8
:091CF500EBF608EAF608E9F62214
:091CFE00EBF0A3EAF0A3E9F022E7
:091D0700EBF208EAF208E9F2220D
:00000001FF
